 i2c

 Timestamp is 4da2a50a (Mon Apr 11 18:51:54 2011)

 Preferred load address is 10000000

 Start         Length     Name                   Class
 0001:00000000 00000004H .CRT$XCA                CODE
 0001:00000004 00000004H .CRT$XCZ                CODE
 0001:00000008 00000004H .CRT$XIA                CODE
 0001:0000000c 00000004H .CRT$XIZ                CODE
 0001:00000010 00000004H .CRT$XPA                CODE
 0001:00000014 00000004H .CRT$XPZ                CODE
 0001:00000018 00000004H .CRT$XTA                CODE
 0001:0000001c 00000004H .CRT$XTZ                CODE
 0001:00000020 00003164H .rdata                  CODE
 0001:00003184 00000020H .rdata$debug            CODE
 0001:000031a4 00009120H .text                   CODE
 0001:0000c2c4 00000048H .xdata                  CODE
 0001:0000c30c 0000003cH .idata$2                CODE
 0001:0000c348 00000014H .idata$3                CODE
 0001:0000c35c 000000d8H .idata$4                CODE
 0001:0000c434 0000008eH .idata$6                CODE
 0001:0000c4d0 000000ffH .edata                  CODE
 0002:00000000 000000d8H .idata$5                DATA
 0002:000000d8 0000044cH .data                   DATA
 0002:00000524 00000010H .bss                    DATA
 0003:00000000 000002a8H .pdata                  DATA

  Address         Publics by Value              Rva+Base       Lib:Object

 0000:00000000       ___safe_se_handler_count   00000000     <absolute>
 0000:00000000       ___safe_se_handler_table   00000000     <absolute>
 0001:00000000       __xc_a                     10001000     corelib0:crt0init.obj
 0001:00000004       __xc_z                     10001004     corelib0:crt0init.obj
 0001:00000008       __xi_a                     10001008     corelib0:crt0init.obj
 0001:0000000c       __xi_z                     1000100c     corelib0:crt0init.obj
 0001:00000010       __xp_a                     10001010     corelib0:crt0init.obj
 0001:00000014       __xp_z                     10001014     corelib0:crt0init.obj
 0001:00000018       __xt_a                     10001018     corelib0:crt0init.obj
 0001:0000001c       __xt_z                     1000101c     corelib0:crt0init.obj
 0001:0000003c       ??_C@_1DG@FMDBLGEG@?$AAI?$AAn?$AAv?$AAa?$AAl?$AAi?$AAd?$AA?5?$AAI?$AA2?$AAC?$AA?5?$AAm?$AAo?$AAd?$AAu?$AAl?$AAe?$AA?5?$AAi?$AAn?$AAd?$AAe?$AAx?$AA?$AN?$AA?6?$AA?$AA@ 1000103c     bspi2c.obj
 0001:00000074       ??_C@_1CO@BGJONOEJ@?$AAI?$AA2?$AAC?$AA_?$AAI?$AAn?$AAi?$AAt?$AA?5?$AA?9?$AA?5?$AAh?$AAD?$AAe?$AAv?$AA?$DN?$AA0?$AAx?$AA?$CF?$AAx?$AA?$AN?$AA?6?$AA?$AA@ 10001074     i2c_mx25_topaz_v1:i2c_io.obj
 0001:000000a8       ??_C@_1EK@OEFBDGBA@?$AAI?$AA2?$AAC?$AA_?$AAI?$AAn?$AAi?$AAt?$AA?3?$AA?5?$AAI?$AA2?$AAC?$AA?5?$AAC?$AAl?$AAa?$AAs?$AAs?$AA?5?$AAF?$AAa?$AAi?$AAl?$AAe?$AAd?$AA?$CB?$AA?5?$AAE?$AAr?$AAr?$AA?$DN@ 100010a8     i2c_mx25_topaz_v1:i2c_io.obj
 0001:000000f8       ??_C@_1EO@DBAJGMMP@?$AAI?$AA2?$AAC?$AA_?$AAI?$AAn?$AAi?$AAt?$AA?3?$AA?5?$AA?5?$AAR?$AAe?$AAg?$AAQ?$AAu?$AAe?$AAr?$AAy?$AAV?$AAa?$AAl?$AAu?$AAe?$AAE?$AAx?$AA?5?$AAf?$AAa?$AAi?$AAl?$AAe@ 100010f8     i2c_mx25_topaz_v1:i2c_io.obj
 0001:00000148       ??_C@_1M@EENNDIOJ@?$AAI?$AAn?$AAd?$AAe?$AAx?$AA?$AA@ 10001148     i2c_mx25_topaz_v1:i2c_io.obj
 0001:00000158       ??_C@_1EK@KPBIOMKA@?$AAI?$AA2?$AAC?$AA_?$AAI?$AAn?$AAi?$AAt?$AA?3?$AA?5?$AA?5?$AAO?$AAp?$AAe?$AAn?$AAD?$AAe?$AAv?$AAi?$AAc?$AAe?$AAK?$AAe?$AAy?$AA?5?$AAf?$AAa?$AAi?$AAl?$AAe?$AAd?$AA?$CB@ 10001158     i2c_mx25_topaz_v1:i2c_io.obj
 0001:000001a4       ??_C@_1BK@ECAEECDB@?$AAI?$AA2?$AAC?$AA_?$AAI?$AAn?$AAi?$AAt?$AA?5?$AA?$CL?$AA?$AN?$AA?6?$AA?$AA@ 100011a4     i2c_mx25_topaz_v1:i2c_io.obj
 0001:000001c0       ??_C@_1BO@COCIDAIB@?$AAI?$AA2?$AAC?$AA_?$AAD?$AAe?$AAi?$AAn?$AAi?$AAt?$AA?5?$AA?9?$AA?$AN?$AA?6?$AA?$AA@ 100011c0     i2c_mx25_topaz_v1:i2c_io.obj
 0001:000001e0       ??_C@_1EC@HCPAPDKB@?$AAI?$AA2?$AAC?$AA_?$AAD?$AAe?$AAi?$AAn?$AAi?$AAt?$AA?5?$AA?$CL?$AAD?$AAe?$AAv?$AAi?$AAc?$AAe?$AAC?$AAo?$AAn?$AAt?$AAe?$AAx?$AAt?$AA?$DN?$AA0?$AAx?$AA?$CF?$AAx?$AA?$AN?$AA?6@ 100011e0     i2c_mx25_topaz_v1:i2c_io.obj
 0001:00000224       ??_C@_1BK@IAGIKLLG@?$AAI?$AA2?$AAC?$AA_?$AAO?$AAp?$AAe?$AAn?$AA?5?$AA?9?$AA?$AN?$AA?6?$AA?$AA@ 10001224     i2c_mx25_topaz_v1:i2c_io.obj
 0001:00000240       ??_C@_1EA@IMBGDPHH@?$AAI?$AA2?$AAC?$AA_?$AAO?$AAp?$AAe?$AAn?$AA?5?$AA?$CL?$AAh?$AAD?$AAe?$AAv?$AAi?$AAc?$AAe?$AAC?$AAo?$AAn?$AAt?$AAe?$AAx?$AAt?$AA?$DN?$AA0?$AAx?$AA?$CF?$AAx?$AA?$AN?$AA?6?$AA?$AA@ 10001240     i2c_mx25_topaz_v1:i2c_io.obj
 0001:00000280       ??_C@_1BM@OBPMOEAO@?$AAI?$AA2?$AAC?$AA_?$AAC?$AAl?$AAo?$AAs?$AAe?$AA?5?$AA?9?$AA?$AN?$AA?6?$AA?$AA@ 10001280     i2c_mx25_topaz_v1:i2c_io.obj
 0001:0000029c       ??_C@_1BM@CHJDONIJ@?$AAI?$AA2?$AAC?$AA_?$AAC?$AAl?$AAo?$AAs?$AAe?$AA?5?$AA?$CL?$AA?$AN?$AA?6?$AA?$AA@ 1000129c     i2c_mx25_topaz_v1:i2c_io.obj
 0001:000002b8       ??_C@_1CE@FAJJIBKD@?$AAI?$AA2?$AAC?$AA_?$AAI?$AAO?$AAC?$AAo?$AAn?$AAt?$AAr?$AAo?$AAl?$AA?5?$AA?9?$AA?$AN?$AA?6?$AA?$AA@ 100012b8     i2c_mx25_topaz_v1:i2c_io.obj
 0001:000002e0       ??_C@_1FK@FLBIPJMP@?$AAE?$AAx?$AAc?$AAe?$AAp?$AAt?$AAi?$AAo?$AAn?$AA?5?$AAi?$AAn?$AA?5?$AAC?$AAS?$AAP?$AAI?$AA?5?$AAI?$AAO?$AAC?$AAT?$AAL?$AA_?$AAP?$AAO?$AAW?$AAE?$AAR?$AA_?$AAC?$AAA@ 100012e0     i2c_mx25_topaz_v1:i2c_io.obj
 0001:0000033c       ??_C@_1CI@OHCJFJPM@?$AAE?$AAR?$AAR?$AAO?$AAR?$AA?3?$AA?5?$AA?$CF?$AAs?$AA?5?$AAl?$AAi?$AAn?$AAe?$AA?5?$AA?$CF?$AAd?$AA?3?$AA?5?$AA?$AA@ 1000133c     i2c_mx25_topaz_v1:i2c_io.obj
 0001:00000368       ??_C@_1LA@GFCDDEBO@?$AAc?$AA?3?$AA?2?$AAw?$AAi?$AAn?$AAc?$AAe?$AAr?$AAo?$AAo?$AAt?$AAs?$AA?2?$AAt?$AAo?$AAp?$AAa?$AAz?$AA?2?$AAw?$AAi?$AAn?$AAc?$AAe?$AA7?$AA0?$AA0?$AA?2?$AAp?$AAl?$AAa@ 10001368     i2c_mx25_topaz_v1:i2c_io.obj
 0001:00000418       ??_C@_1DA@MHMGIHOO@?$AAI?$AA2?$AAC?$AA_?$AAI?$AAO?$AAC?$AAo?$AAn?$AAt?$AAr?$AAo?$AAl?$AA?3?$AAR?$AAE?$AAS?$AAE?$AAT?$AA?5?$AA?9?$AA?$AN?$AA?6?$AA?$AA@ 10001418     i2c_mx25_topaz_v1:i2c_io.obj
 0001:00000448       ??_C@_1DA@BKJIOGJ@?$AAI?$AA2?$AAC?$AA_?$AAI?$AAO?$AAC?$AAo?$AAn?$AAt?$AAr?$AAo?$AAl?$AA?3?$AAR?$AAE?$AAS?$AAE?$AAT?$AA?5?$AA?$CL?$AA?$AN?$AA?6?$AA?$AA@ 10001448     i2c_mx25_topaz_v1:i2c_io.obj
 0001:00000478       ??_C@_1EK@EGBHBCGP@?$AAI?$AA2?$AAC?$AA_?$AAI?$AAO?$AAC?$AAo?$AAn?$AAt?$AAr?$AAo?$AAl?$AA?3?$AAI?$AA2?$AAC?$AA_?$AAI?$AAO?$AAC?$AAT?$AAL?$AA_?$AAT?$AAR?$AAA?$AAN?$AAS?$AAF?$AAE?$AAR@ 10001478     i2c_mx25_topaz_v1:i2c_io.obj
 0001:000004c8       ??_C@_1FC@HNNCAIOH@?$AAI?$AA2?$AAC?$AA_?$AAI?$AAO?$AAC?$AAo?$AAn?$AAt?$AAr?$AAo?$AAl?$AA?3?$AAG?$AAE?$AAT?$AA_?$AAS?$AAE?$AAL?$AAF?$AA_?$AAA?$AAD?$AAD?$AAR?$AA?5?$AA?9?$AA?5?$AAV?$AAa@ 100014c8     i2c_mx25_topaz_v1:i2c_io.obj
 0001:00000520       ??_C@_1EA@HOENNIME@?$AAI?$AA2?$AAC?$AA_?$AAI?$AAO?$AAC?$AAo?$AAn?$AAt?$AAr?$AAo?$AAl?$AA?3?$AAG?$AAE?$AAT?$AA_?$AAS?$AAE?$AAL?$AAF?$AA_?$AAA?$AAD?$AAD?$AAR?$AA?5?$AA?$CL?$AA?$AN?$AA?6?$AA?$AA@ 10001520     i2c_mx25_topaz_v1:i2c_io.obj
 0001:00000560       ??_C@_1FG@NLOMNKA@?$AAI?$AA2?$AAC?$AA_?$AAI?$AAO?$AAC?$AAo?$AAn?$AAt?$AAr?$AAo?$AAl?$AA?3?$AAS?$AAE?$AAT?$AA_?$AAS?$AAE?$AAL?$AAF?$AA_?$AAA?$AAD?$AAD?$AAR?$AA?5?$AA?$CL?$AA?5?$AAV?$AAa@ 10001560     i2c_mx25_topaz_v1:i2c_io.obj
 0001:000005b8       ??_C@_1IC@KHAIPPEI@?$AAI?$AA2?$AAC?$AA_?$AAI?$AAO?$AAC?$AAo?$AAn?$AAt?$AAr?$AAo?$AAl?$AA?3?$AA?5?$AAI?$AA2?$AAC?$AA?5?$AAf?$AAr?$AAe?$AAq?$AAu?$AAe?$AAn?$AAc?$AAy?$AA?5?$AAm?$AAa?$AAy@ 100015b8     i2c_mx25_topaz_v1:i2c_io.obj
 0001:00000640       ??_C@_1FG@NAPOACDN@?$AAI?$AA2?$AAC?$AA_?$AAI?$AAO?$AAC?$AAo?$AAn?$AAt?$AAr?$AAo?$AAl?$AA?3?$AAS?$AAE?$AAT?$AA_?$AAF?$AAR?$AAE?$AAQ?$AAU?$AAE?$AAN?$AAC?$AAY?$AA?5?$AA?$CL?$AA?5?$AAV?$AAa@ 10001640     i2c_mx25_topaz_v1:i2c_io.obj
 0001:00000698       ??_C@_1FI@ELEHJNIJ@?$AAI?$AA2?$AAC?$AA_?$AAI?$AAO?$AAC?$AAo?$AAn?$AAt?$AAr?$AAo?$AAl?$AA?3?$AAS?$AAE?$AAT?$AA_?$AAC?$AAL?$AAO?$AAC?$AAK?$AA_?$AAR?$AAA?$AAT?$AAE?$AA?5?$AA?$CL?$AA?5?$AAV@ 10001698     i2c_mx25_topaz_v1:i2c_io.obj
 0001:000006f0       ??_C@_1FE@CCKAONLP@?$AAI?$AA2?$AAC?$AA_?$AAI?$AAO?$AAC?$AAo?$AAn?$AAt?$AAr?$AAo?$AAl?$AA?3?$AAG?$AAE?$AAT?$AA_?$AAC?$AAL?$AAO?$AAC?$AAK?$AA_?$AAR?$AAA?$AAT?$AAE?$AA?5?$AA?9?$AA?5?$AAV@ 100016f0     i2c_mx25_topaz_v1:i2c_io.obj
 0001:00000748       ??_C@_1EC@OKIABNEK@?$AAI?$AA2?$AAC?$AA_?$AAI?$AAO?$AAC?$AAo?$AAn?$AAt?$AAr?$AAo?$AAl?$AA?3?$AAG?$AAE?$AAT?$AA_?$AAC?$AAL?$AAO?$AAC?$AAK?$AA_?$AAR?$AAA?$AAT?$AAE?$AA?5?$AA?$CL?$AA?$AN?$AA?6@ 10001748     i2c_mx25_topaz_v1:i2c_io.obj
 0001:00000790       ??_C@_1EI@DLMELBOO@?$AAI?$AA2?$AAC?$AA_?$AAI?$AAO?$AAC?$AAo?$AAn?$AAt?$AAr?$AAo?$AAl?$AA?3?$AAI?$AAS?$AA_?$AAS?$AAL?$AAA?$AAV?$AAE?$AA?5?$AA?9?$AA?5?$AAV?$AAa?$AAl?$AA?$DN?$AA0?$AAx?$AA?$CF@ 10001790     i2c_mx25_topaz_v1:i2c_io.obj
 0001:000007d8       ??_C@_1DG@LJJAKLMJ@?$AAI?$AA2?$AAC?$AA_?$AAI?$AAO?$AAC?$AAo?$AAn?$AAt?$AAr?$AAo?$AAl?$AA?3?$AAI?$AAS?$AA_?$AAS?$AAL?$AAA?$AAV?$AAE?$AA?5?$AA?$CL?$AA?$AN?$AA?6?$AA?$AA@ 100017d8     i2c_mx25_topaz_v1:i2c_io.obj
 0001:00000810       ??_C@_1EK@GBPPHJBK@?$AAI?$AA2?$AAC?$AA_?$AAI?$AAO?$AAC?$AAo?$AAn?$AAt?$AAr?$AAo?$AAl?$AA?3?$AAI?$AAS?$AA_?$AAM?$AAA?$AAS?$AAT?$AAE?$AAR?$AA?5?$AA?9?$AA?5?$AAV?$AAa?$AAl?$AA?$DN?$AA0?$AAx@ 10001810     i2c_mx25_topaz_v1:i2c_io.obj
 0001:0000085c       ??_C@_1DI@FOMPNCPC@?$AAI?$AA2?$AAC?$AA_?$AAI?$AAO?$AAC?$AAo?$AAn?$AAt?$AAr?$AAo?$AAl?$AA?3?$AAI?$AAS?$AA_?$AAM?$AAA?$AAS?$AAT?$AAE?$AAR?$AA?5?$AA?$CL?$AA?$AN?$AA?6?$AA?$AA@ 1000185c     i2c_mx25_topaz_v1:i2c_io.obj
 0001:00000898       ??_C@_1EE@GOJPLBJJ@?$AAI?$AA2?$AAC?$AA_?$AAI?$AAO?$AAC?$AAo?$AAn?$AAt?$AAr?$AAo?$AAl?$AA?3?$AAS?$AAE?$AAT?$AA_?$AAM?$AAA?$AAS?$AAT?$AAE?$AAR?$AA_?$AAM?$AAO?$AAD?$AAE?$AA?5?$AA?$CL?$AA?$AN@ 10001898     i2c_mx25_topaz_v1:i2c_io.obj
 0001:000008e0       ??_C@_1EC@BKOABMJG@?$AAI?$AA2?$AAC?$AA_?$AAI?$AAO?$AAC?$AAo?$AAn?$AAt?$AAr?$AAo?$AAl?$AA?3?$AAS?$AAE?$AAT?$AA_?$AAS?$AAL?$AAA?$AAV?$AAE?$AA_?$AAM?$AAO?$AAD?$AAE?$AA?5?$AA?9?$AA?$AN?$AA?6@ 100018e0     i2c_mx25_topaz_v1:i2c_io.obj
 0001:00000928       ??_C@_1EC@NMIPBFBB@?$AAI?$AA2?$AAC?$AA_?$AAI?$AAO?$AAC?$AAo?$AAn?$AAt?$AAr?$AAo?$AAl?$AA?3?$AAS?$AAE?$AAT?$AA_?$AAS?$AAL?$AAA?$AAV?$AAE?$AA_?$AAM?$AAO?$AAD?$AAE?$AA?5?$AA?$CL?$AA?$AN?$AA?6@ 10001928     i2c_mx25_topaz_v1:i2c_io.obj
 0001:00000970       ??_C@_1EI@DONFLMGA@?$AAI?$AA2?$AAC?$AA_?$AAI?$AAO?$AAC?$AAo?$AAn?$AAt?$AAr?$AAo?$AAl?$AA?3?$AA?5?$AA?$CL?$AAh?$AAO?$AAp?$AAe?$AAn?$AAC?$AAo?$AAn?$AAt?$AAe?$AAx?$AAt?$AA?$DN?$AA0?$AAx?$AA?$CF@ 10001970     i2c_mx25_topaz_v1:i2c_io.obj
 0001:000009b8       ??_C@_1GK@FJAEABEO@?$AAI?$AA2?$AAC?$AA_?$AAD?$AAl?$AAl?$AAE?$AAn?$AAt?$AAr?$AAy?$AA?3?$AA?5?$AAD?$AAL?$AAL?$AA_?$AAP?$AAR?$AAO?$AAC?$AAE?$AAS?$AAS?$AA_?$AAD?$AAE?$AAT?$AAA?$AAC?$AAH@ 100019b8     i2c_mx25_topaz_v1:i2c_io.obj
 0001:00000a28       ??_C@_1GK@BNIBCNLI@?$AAI?$AA2?$AAC?$AA_?$AAD?$AAl?$AAl?$AAE?$AAn?$AAt?$AAr?$AAy?$AA?3?$AA?5?$AAD?$AAL?$AAL?$AA_?$AAP?$AAR?$AAO?$AAC?$AAE?$AAS?$AAS?$AA_?$AAA?$AAT?$AAT?$AAA?$AAC?$AAH@ 10001a28     i2c_mx25_topaz_v1:i2c_io.obj
 0001:00000a94       ??_7?$Buffer_t@VDuplicateTraits_t@detail@marshal@ce@@@detail@marshal@ce@@6B@ 10001a94     i2c_mx25_topaz_v1:i2c_io.obj
 0001:00000b18       ??_C@_1CO@LCLKJFDO@?$AAI?$AA2?$AAC?$AAC?$AAl?$AAa?$AAs?$AAs?$AA?3?$AA?3?$AAI?$AA2?$AAC?$AAC?$AAl?$AAa?$AAs?$AAs?$AA?5?$AA?9?$AA?$AN?$AA?6?$AA?$AA@ 10001b18     i2c_mx25_topaz_v1:i2cClass.obj
 0001:00000b48       ??_C@_1FM@JOBMIHOG@?$AAI?$AA2?$AAC?$AAC?$AAl?$AAa?$AAs?$AAs?$AA?3?$AA?3?$AAI?$AA2?$AAC?$AAC?$AAl?$AAa?$AAs?$AAs?$AA?3?$AA?5?$AAD?$AAe?$AAf?$AAa?$AAu?$AAl?$AAt?$AA?5?$AAt?$AAo?$AA?5?$AAM@ 10001b48     i2c_mx25_topaz_v1:i2cClass.obj
 0001:00000ba8       ??_C@_1FO@BIKBBCID@?$AAI?$AA2?$AAC?$AAC?$AAl?$AAa?$AAs?$AAs?$AA?3?$AA?3?$AAI?$AA2?$AAC?$AAC?$AAl?$AAa?$AAs?$AAs?$AA?3?$AAI?$AA2?$AAC?$AA_?$AAW?$AAO?$AAR?$AAD?$AA_?$AAO?$AAU?$AAT?$AA?$CI@ 10001ba8     i2c_mx25_topaz_v1:i2cClass.obj
 0001:00000c08       ??_C@_1FO@MOANANJB@?$AA?$CF?$AAs?$AA?3?$AA?5?$AAc?$AAr?$AAe?$AAa?$AAt?$AAe?$AA?5?$AAI?$AA2?$AAC?$AA?5?$AAI?$AAS?$AAT?$AA?5?$AAt?$AAh?$AAr?$AAe?$AAa?$AAd?$AA?5?$AAs?$AAu?$AAc?$AAc?$AAe?$AAs@ 10001c08     i2c_mx25_topaz_v1:i2cClass.obj
 0001:00000c68       ??_C@_1EI@LJIGNOLF@?$AA?$CF?$AAs?$AA?3?$AA?5?$AAc?$AAr?$AAe?$AAa?$AAt?$AAe?$AA?5?$AAI?$AA2?$AAC?$AA?5?$AAI?$AAS?$AAT?$AA?5?$AAt?$AAh?$AAr?$AAe?$AAa?$AAd?$AA?5?$AAs?$AAu?$AAc?$AAc?$AAe?$AAs@ 10001c68     i2c_mx25_topaz_v1:i2cClass.obj
 0001:00000cb0       ??_C@_1DG@IKMOEBDF@?$AA?$CF?$AAs?$AA?3?$AA?5?$AAC?$AAr?$AAe?$AAa?$AAt?$AAe?$AAT?$AAh?$AAr?$AAe?$AAa?$AAd?$AA?5?$AAf?$AAa?$AAi?$AAl?$AAe?$AAd?$AA?$CB?$AA?$AN?$AA?6?$AA?$AA@ 10001cb0     i2c_mx25_topaz_v1:i2cClass.obj
 0001:00000ce8       ??_C@_1HO@KLJIHGDF@?$AAI?$AA2?$AAC?$AAC?$AAl?$AAa?$AAs?$AAs?$AA?3?$AA?3?$AAI?$AA2?$AAC?$AAC?$AAl?$AAa?$AAs?$AAs?$AA?3?$AAB?$AAS?$AAP?$AAG?$AAe?$AAt?$AAT?$AAi?$AAm?$AAe?$AAo?$AAu?$AAt@ 10001ce8     i2c_mx25_topaz_v1:i2cClass.obj
 0001:00000d68       ??_C@_1HK@EJLDMDJF@?$AAI?$AA2?$AAC?$AAC?$AAl?$AAa?$AAs?$AAs?$AA?3?$AA?3?$AAI?$AA2?$AAC?$AAC?$AAl?$AAa?$AAs?$AAs?$AA?3?$AAI?$AAn?$AAt?$AAe?$AAr?$AAr?$AAu?$AAp?$AAt?$AAi?$AAn?$AAi?$AAt@ 10001d68     i2c_mx25_topaz_v1:i2cClass.obj
 0001:00000de8       ??_C@_1JA@FKDODFOK@?$AAI?$AA2?$AAC?$AAC?$AAl?$AAa?$AAs?$AAs?$AA?3?$AA?3?$AAI?$AA2?$AAC?$AAC?$AAl?$AAa?$AAs?$AAs?$AA?3?$AAI?$AAn?$AAt?$AAe?$AAr?$AAr?$AAu?$AAp?$AAt?$AAi?$AAn?$AAi?$AAt@ 10001de8     i2c_mx25_topaz_v1:i2cClass.obj
 0001:00000e78       ??_C@_1HA@IEPKFPCI@?$AAI?$AA2?$AAC?$AAC?$AAl?$AAa?$AAs?$AAs?$AA?3?$AA?3?$AAI?$AA2?$AAC?$AAC?$AAl?$AAa?$AAs?$AAs?$AA?3?$AAK?$AAe?$AAr?$AAn?$AAe?$AAl?$AAI?$AAo?$AAC?$AAo?$AAn?$AAt?$AAr@ 10001e78     i2c_mx25_topaz_v1:i2cClass.obj
 0001:00000ee8       ??_C@_1JG@MMOGEJFA@?$AAI?$AA2?$AAC?$AAC?$AAl?$AAa?$AAs?$AAs?$AA?3?$AA?3?$AAI?$AA2?$AAC?$AAC?$AAl?$AAa?$AAs?$AAs?$AA?3?$AAK?$AAe?$AAr?$AAn?$AAe?$AAl?$AAI?$AAo?$AAC?$AAo?$AAn?$AAt?$AAr@ 10001ee8     i2c_mx25_topaz_v1:i2cClass.obj
 0001:00000f80       ??_C@_1KM@MDDELGGK@?$AAI?$AA2?$AAC?$AAC?$AAl?$AAa?$AAs?$AAs?$AA?3?$AA?3?$AAI?$AA2?$AAC?$AAC?$AAl?$AAa?$AAs?$AAs?$AA?3?$AAI?$AAn?$AAi?$AAt?$AAi?$AAa?$AAl?$AAi?$AAz?$AAe?$AAC?$AAr?$AAi@ 10001f80     i2c_mx25_topaz_v1:i2cClass.obj
 0001:00001030       ??_C@_1EO@GJHDEMOE@?$AA?$CF?$AAs?$AA?3?$AA?5?$AAE?$AAr?$AAr?$AAo?$AAr?$AA?5?$AAc?$AAo?$AAn?$AAf?$AAi?$AAg?$AAu?$AAr?$AAi?$AAn?$AAg?$AA?5?$AAI?$AAO?$AAM?$AAU?$AAX?$AA?5?$AAf?$AAo?$AAr?$AA?5@ 10002030     i2c_mx25_topaz_v1:i2cClass.obj
 0001:00001080       ??_C@_1CG@FILMNMOG@?$AAI?$AA2?$AAC?$AAC?$AAl?$AAa?$AAs?$AAs?$AA?3?$AA?3?$AAI?$AA2?$AAC?$AAC?$AAl?$AAa?$AAs?$AAs?$AA?$AA@ 10002080     i2c_mx25_topaz_v1:i2cClass.obj
 0001:000010a8       ??_C@_1LI@MHFLBAJK@?$AAI?$AA2?$AAC?$AAC?$AAl?$AAa?$AAs?$AAs?$AA?3?$AA?3?$AAI?$AA2?$AAC?$AAC?$AAl?$AAa?$AAs?$AAs?$AA?3?$AAI?$AAn?$AAi?$AAt?$AAi?$AAa?$AAl?$AAi?$AAz?$AAe?$AAC?$AAr?$AAi@ 100020a8     i2c_mx25_topaz_v1:i2cClass.obj
 0001:00001160       ??_C@_1CA@IODADCHB@?$AAE?$AAV?$AAE?$AAN?$AAT?$AA_?$AAI?$AA2?$AAC?$AA3?$AAS?$AAL?$AAA?$AAV?$AAE?$AA?$AA@ 10002160     i2c_mx25_topaz_v1:i2cClass.obj
 0001:00001180       ??_C@_1CA@BDDPNDAH@?$AAE?$AAV?$AAE?$AAN?$AAT?$AA_?$AAI?$AA2?$AAC?$AA2?$AAS?$AAL?$AAA?$AAV?$AAE?$AA?$AA@ 10002180     i2c_mx25_topaz_v1:i2cClass.obj
 0001:000011a0       ??_C@_1CA@GPFOPGNM@?$AAE?$AAV?$AAE?$AAN?$AAT?$AA_?$AAI?$AA2?$AAC?$AA1?$AAS?$AAL?$AAA?$AAV?$AAE?$AA?$AA@ 100021a0     i2c_mx25_topaz_v1:i2cClass.obj
 0001:000011c0       ??_C@_1HE@GDDOFFBJ@?$AAI?$AA2?$AAC?$AAC?$AAl?$AAa?$AAs?$AAs?$AA?3?$AA?3?$AAI?$AA2?$AAC?$AAC?$AAl?$AAa?$AAs?$AAs?$AA?3?$AAC?$AAr?$AAe?$AAa?$AAt?$AAe?$AAE?$AAv?$AAe?$AAn?$AAt?$AA?$CI?$AA?$CJ@ 100021c0     i2c_mx25_topaz_v1:i2cClass.obj
 0001:00001238       ??_C@_1LM@EFJNLIGI@?$AAI?$AA2?$AAC?$AAC?$AAl?$AAa?$AAs?$AAs?$AA?3?$AA?3?$AAI?$AA2?$AAC?$AAC?$AAl?$AAa?$AAs?$AAs?$AA?3?$AAC?$AAr?$AAe?$AAa?$AAt?$AAe?$AAE?$AAv?$AAe?$AAn?$AAt?$AA?$CI?$AA?$CJ@ 10002238     i2c_mx25_topaz_v1:i2cClass.obj
 0001:000012f8       ??_C@_1GO@NLKHDBEJ@?$AAI?$AA2?$AAC?$AAC?$AAl?$AAa?$AAs?$AAs?$AA?3?$AA?3?$AAI?$AA2?$AAC?$AAC?$AAl?$AAa?$AAs?$AAs?$AA?3?$AAC?$AAr?$AAe?$AAa?$AAt?$AAe?$AAE?$AAv?$AAe?$AAn?$AAt?$AA?$CI?$AA?$CJ@ 100022f8     i2c_mx25_topaz_v1:i2cClass.obj
 0001:00001368       ??_C@_1LM@HALIBCHD@?$AAI?$AA2?$AAC?$AAC?$AAl?$AAa?$AAs?$AAs?$AA?3?$AA?3?$AAI?$AA2?$AAC?$AAC?$AAl?$AAa?$AAs?$AAs?$AA?3?$AAC?$AAr?$AAe?$AAa?$AAt?$AAe?$AAE?$AAv?$AAe?$AAn?$AAt?$AA?$CI?$AA?$CJ@ 10002368     i2c_mx25_topaz_v1:i2cClass.obj
 0001:00001428       ??_C@_1GG@LOCNNAFI@?$AAI?$AA2?$AAC?$AAC?$AAl?$AAa?$AAs?$AAs?$AA?3?$AA?3?$AAI?$AA2?$AAC?$AAC?$AAl?$AAa?$AAs?$AAs?$AA?3?$AAM?$AAm?$AAM?$AAa?$AAp?$AAI?$AAo?$AAS?$AAp?$AAa?$AAc?$AAe?$AA?$CI@ 10002428     i2c_mx25_topaz_v1:i2cClass.obj
 0001:00001490       ??_C@_1HC@POEDKKJM@?$AAI?$AA2?$AAC?$AAC?$AAl?$AAa?$AAs?$AAs?$AA?3?$AA?3?$AAI?$AA2?$AAC?$AAC?$AAl?$AAa?$AAs?$AAs?$AA?3?$AAM?$AAm?$AAM?$AAa?$AAp?$AAI?$AAo?$AAS?$AAp?$AAa?$AAc?$AAe?$AA?$CI@ 10002490     i2c_mx25_topaz_v1:i2cClass.obj
 0001:00001504       ??_C@_1CO@HENFJMLJ@?$AAI?$AA2?$AAC?$AAC?$AAl?$AAa?$AAs?$AAs?$AA?3?$AA?3?$AAI?$AA2?$AAC?$AAC?$AAl?$AAa?$AAs?$AAs?$AA?5?$AA?$CL?$AA?$AN?$AA?6?$AA?$AA@ 10002504     i2c_mx25_topaz_v1:i2cClass.obj
 0001:00001534       ??_C@_1DA@EJLEFIKO@?$AAI?$AA2?$AAC?$AAC?$AAl?$AAa?$AAs?$AAs?$AA?3?$AA?3?$AA?$HO?$AAI?$AA2?$AAC?$AAC?$AAl?$AAa?$AAs?$AAs?$AA?5?$AA?9?$AA?$AN?$AA?6?$AA?$AA@ 10002534     i2c_mx25_topaz_v1:i2cClass.obj
 0001:00001568       ??_C@_1JA@HAIFHFLM@?$AAI?$AA2?$AAC?$AAC?$AAl?$AAa?$AAs?$AAs?$AA?3?$AA?3?$AA?$HO?$AAI?$AA2?$AAC?$AAC?$AAl?$AAa?$AAs?$AAs?$AA?3?$AA?5?$AAR?$AAe?$AAl?$AAe?$AAa?$AAs?$AAe?$AA?5?$AAI?$AA2?$AAC@ 10002568     i2c_mx25_topaz_v1:i2cClass.obj
 0001:000015f8       ??_C@_1HE@IPMPHGMB@?$AAI?$AA2?$AAC?$AAC?$AAl?$AAa?$AAs?$AAs?$AA?3?$AA?3?$AA?$HO?$AAI?$AA2?$AAC?$AAC?$AAl?$AAa?$AAs?$AAs?$AA?3?$AA?5?$AAR?$AAe?$AAl?$AAe?$AAa?$AAs?$AAe?$AA?5?$AAI?$AAn?$AAt@ 100025f8     i2c_mx25_topaz_v1:i2cClass.obj
 0001:00001670       ??_C@_1LC@LHDEFGDE@?$AAI?$AA2?$AAC?$AAC?$AAl?$AAa?$AAs?$AAs?$AA?3?$AA?3?$AA?$HO?$AAI?$AA2?$AAC?$AAC?$AAl?$AAa?$AAs?$AAs?$AA?3?$AAD?$AAe?$AAl?$AAe?$AAt?$AAe?$AAC?$AAr?$AAi?$AAt?$AAi?$AAc@ 10002670     i2c_mx25_topaz_v1:i2cClass.obj
 0001:00001728       ??_C@_1EM@HCNAFH@?$AAE?$AAR?$AAR?$AAO?$AAR?$AA?3?$AA?5?$AAF?$AAa?$AAi?$AAl?$AAe?$AAd?$AA?5?$AAt?$AAo?$AA?5?$AAr?$AAe?$AAl?$AAe?$AAa?$AAs?$AAe?$AA?5?$AAd?$AAw?$AAS?$AAy?$AAs?$AAI?$AAn@ 10002728     i2c_mx25_topaz_v1:i2cClass.obj
 0001:00001778       ??_C@_1GK@DCLJCPBJ@?$AAI?$AA2?$AAC?$AAC?$AAl?$AAa?$AAs?$AAs?$AA?3?$AA?3?$AA?$HO?$AAI?$AA2?$AAC?$AAC?$AAl?$AAa?$AAs?$AAs?$AA?$CI?$AA?$CJ?$AA?3?$AA?5?$AAR?$AAe?$AAl?$AAe?$AAa?$AAs?$AAi?$AAn?$AAg@ 10002778     i2c_mx25_topaz_v1:i2cClass.obj
 0001:000017e8       ??_C@_1GC@PFGIPEEG@?$AAI?$AA2?$AAC?$AAC?$AAl?$AAa?$AAs?$AAs?$AA?3?$AA?3?$AA?$HO?$AAI?$AA2?$AAC?$AAC?$AAl?$AAa?$AAs?$AAs?$AA?3?$AA?5?$AAR?$AAe?$AAl?$AAe?$AAa?$AAs?$AAe?$AA?5?$AAS?$AAy?$AAs@ 100027e8     i2c_mx25_topaz_v1:i2cClass.obj
 0001:0000184c       ??_C@_1DA@IPNLFBCJ@?$AAI?$AA2?$AAC?$AAC?$AAl?$AAa?$AAs?$AAs?$AA?3?$AA?3?$AA?$HO?$AAI?$AA2?$AAC?$AAC?$AAl?$AAa?$AAs?$AAs?$AA?5?$AA?$CL?$AA?$AN?$AA?6?$AA?$AA@ 1000284c     i2c_mx25_topaz_v1:i2cClass.obj
 0001:00001880       ??_C@_1HC@JDDEOKKN@?$AAW?$AAa?$AAr?$AAn?$AAi?$AAn?$AAg?$AA?3?$AA?5?$AAE?$AAv?$AAe?$AAn?$AAt?$AA?5?$AAr?$AAe?$AAm?$AAa?$AAi?$AAn?$AA?5?$AAp?$AAe?$AAn?$AAd?$AAi?$AAn?$AAg?$AA?5?$AAA?$AAF@ 10002880     i2c_mx25_topaz_v1:i2cClass.obj
 0001:000018f4       ??_C@_1CO@CMCFOKNL@?$AAA?$AAd?$AAd?$AAr?$AAe?$AAs?$AAs?$AA?5?$AAc?$AAy?$AAc?$AAl?$AAe?$AA?5?$AAN?$AAo?$AA?5?$AAA?$AAC?$AAK?$AA?$AN?$AA?6?$AA?$AA@ 100028f4     i2c_mx25_topaz_v1:i2cClass.obj
 0001:00001928       ??_C@_1GE@KPHHIAFA@?$AAI?$AA2?$AAC?$AAC?$AAl?$AAa?$AAs?$AAs?$AA?3?$AA?3?$AAG?$AAe?$AAn?$AAe?$AAr?$AAa?$AAt?$AAe?$AAS?$AAt?$AAa?$AAr?$AAt?$AA?$CI?$AA?$CJ?$AA?3?$AA?5?$AAN?$AAo?$AA?5?$AAA?$AAC@ 10002928     i2c_mx25_topaz_v1:i2cClass.obj
 0001:00001990       ??_C@_1NA@LDHNPBLN@?$AAI?$AA2?$AAC?$AAC?$AAl?$AAa?$AAs?$AAs?$AA?3?$AA?3?$AAP?$AAr?$AAo?$AAc?$AAe?$AAs?$AAs?$AAP?$AAa?$AAc?$AAk?$AAe?$AAt?$AA?$CI?$AA?$CJ?$AA?3?$AA?5?$AAT?$AAi?$AAm?$AAe?$AAd@ 10002990     i2c_mx25_topaz_v1:i2cClass.obj
 0001:00001a60       ??_C@_1KK@NCKDPBOF@?$AAI?$AA2?$AAC?$AAC?$AAl?$AAa?$AAs?$AAs?$AA?3?$AA?3?$AAP?$AAr?$AAo?$AAc?$AAe?$AAs?$AAs?$AAP?$AAa?$AAc?$AAk?$AAe?$AAt?$AA?$CI?$AA?$CJ?$AA?3?$AA?5?$AAT?$AAi?$AAm?$AAe?$AAd@ 10002a60     i2c_mx25_topaz_v1:i2cClass.obj
 0001:00001b10       ??_C@_1EM@DIANPGAN@?$AAD?$AAo?$AAw?$AAn?$AA?5?$AAg?$AAr?$AAa?$AAd?$AAe?$AA?5?$AAi?$AA2?$AAc?$AA?5?$AAt?$AAo?$AA?5?$AAp?$AAo?$AAl?$AAl?$AAi?$AAn?$AAg?$AA?5?$AAm?$AAo?$AAd?$AAe?$AA?4?$AA?$CI@ 10002b10     i2c_mx25_topaz_v1:i2cClass.obj
 0001:00001b60       ??_C@_1HM@MIJIGCPD@?$AAI?$AA2?$AAC?$AAC?$AAl?$AAa?$AAs?$AAs?$AA?3?$AA?3?$AAP?$AAr?$AAo?$AAc?$AAe?$AAs?$AAs?$AAP?$AAa?$AAc?$AAk?$AAe?$AAt?$AA?$CI?$AA?$CJ?$AA?3?$AA?5?$AAW?$AAa?$AAi?$AAt?$AAi@ 10002b60     i2c_mx25_topaz_v1:i2cClass.obj
 0001:00001be0       ??_C@_1EK@NDPLKP@?$AAD?$AAo?$AAw?$AAn?$AA?5?$AAg?$AAr?$AAa?$AAd?$AAe?$AA?5?$AAi?$AA2?$AAc?$AA?5?$AAt?$AAo?$AA?5?$AAp?$AAo?$AAl?$AAl?$AAi?$AAn?$AAg?$AA?5?$AAm?$AAo?$AAd?$AAe?$AA?4?$AA?$CI@ 10002be0     i2c_mx25_topaz_v1:i2cClass.obj
 0001:00001c30       ??_C@_1HA@LOOGODDI@?$AAI?$AA2?$AAC?$AAC?$AAl?$AAa?$AAs?$AAs?$AA?3?$AA?3?$AAP?$AAr?$AAo?$AAc?$AAe?$AAs?$AAs?$AAP?$AAa?$AAc?$AAk?$AAe?$AAt?$AA?$CI?$AA?$CJ?$AA?3?$AA?5?$AAT?$AAo?$AA?5?$AAI?$AA2@ 10002c30     i2c_mx25_topaz_v1:i2cClass.obj
 0001:00001ca0       ??_C@_1EK@BIFBBEDO@?$AAI?$AAI?$AAF?$AA?5?$AAc?$AAa?$AAn?$AA?5?$AAn?$AAo?$AAt?$AA?5?$AAr?$AAe?$AAs?$AAe?$AAt?$AA?5?$AAi?$AAn?$AA?5?$AAG?$AAe?$AAn?$AAe?$AAr?$AAa?$AAt?$AAe?$AAS?$AAt?$AAa@ 10002ca0     i2c_mx25_topaz_v1:i2cClass.obj
 0001:00001cf0       ??_C@_1GC@MBOBGOKA@?$AAI?$AA2?$AAC?$AAC?$AAl?$AAa?$AAs?$AAs?$AA?3?$AA?3?$AAP?$AAr?$AAo?$AAc?$AAe?$AAs?$AAs?$AAP?$AAa?$AAc?$AAk?$AAe?$AAt?$AA?$CI?$AA?$CJ?$AA?3?$AA?5?$AAB?$AAu?$AAs?$AA?5?$AAM@ 10002cf0     i2c_mx25_topaz_v1:i2cClass.obj
 0001:00001d54       ??_C@_1DE@BLMFIOMK@?$AAM?$AAa?$AAs?$AAt?$AAe?$AAr?$AA?5?$AAm?$AAo?$AAd?$AAe?$AA?5?$AAs?$AAe?$AAt?$AA?5?$AAf?$AAa?$AAi?$AAl?$AAu?$AAr?$AAe?$AA?$AN?$AA?6?$AA?$AA@ 10002d54     i2c_mx25_topaz_v1:i2cClass.obj
 0001:00001d88       ??_C@_1DM@LKCCLCDD@?$AAI?$AAA?$AAL?$AA?5?$AAd?$AAe?$AAt?$AAe?$AAc?$AAt?$AA?5?$AAi?$AAn?$AA?5?$AAG?$AAe?$AAn?$AAe?$AAr?$AAa?$AAt?$AAe?$AAS?$AAt?$AAa?$AAr?$AAt?$AA?$AN?$AA?6?$AA?$AA@ 10002d88     i2c_mx25_topaz_v1:i2cClass.obj
 0001:00001dc4       ??_C@_1DM@NJJIKKBN@?$AAG?$AAe?$AAn?$AAe?$AAr?$AAa?$AAt?$AAe?$AA?5?$AAS?$AAt?$AAa?$AAr?$AAt?$AA?5?$AAc?$AAa?$AAn?$AA?8?$AAt?$AA?5?$AAl?$AAa?$AAu?$AAn?$AAc?$AAh?$AA?$AN?$AA?6?$AA?$AA@ 10002dc4     i2c_mx25_topaz_v1:i2cClass.obj
 0001:00001e00       ??_C@_1DO@MCKKPKOO@?$AAG?$AAe?$AAn?$AAe?$AAr?$AAa?$AAt?$AAe?$AA?5?$AAS?$AAt?$AAa?$AAr?$AAt?$AA?5?$AAc?$AAa?$AAn?$AA?8?$AAt?$AA?5?$AAb?$AAe?$AA?5?$AAd?$AAo?$AAn?$AAe?$AA?$AN?$AA?6?$AA?$AA@ 10002e00     i2c_mx25_topaz_v1:i2cClass.obj
 0001:00001e40       ??_C@_1EE@HHAOILO@?$AAI?$AAI?$AAF?$AA?5?$AAs?$AAt?$AAi?$AAl?$AAl?$AA?5?$AAp?$AAe?$AAn?$AAd?$AA?5?$AAi?$AAn?$AA?5?$AAG?$AAe?$AAn?$AAe?$AAr?$AAa?$AAt?$AAe?$AAS?$AAt?$AAa?$AAr?$AAt?$AA?$AN@ 10002e40     i2c_mx25_topaz_v1:i2cClass.obj
 0001:00001e88       ??_C@_1EO@JLNKKEBM@?$AAD?$AAo?$AAw?$AAn?$AA?5?$AAg?$AAr?$AAa?$AAd?$AAe?$AA?5?$AAi?$AA2?$AAc?$AA?5?$AAt?$AAo?$AA?5?$AAp?$AAo?$AAl?$AAl?$AAi?$AAn?$AAg?$AA?5?$AAm?$AAo?$AAd?$AAe?$AA?4?$AA?$CI@ 10002e88     i2c_mx25_topaz_v1:i2cClass.obj
 0001:00001ed8       ??_C@_1EM@DJOHGNPP@?$AAD?$AAo?$AAw?$AAn?$AA?5?$AAg?$AAr?$AAa?$AAd?$AAe?$AA?5?$AAi?$AA2?$AAc?$AA?5?$AAt?$AAo?$AA?5?$AAp?$AAo?$AAl?$AAl?$AAi?$AAn?$AAg?$AA?5?$AAm?$AAo?$AAd?$AAe?$AA?4?$AA?$CI@ 10002ed8     i2c_mx25_topaz_v1:i2cClass.obj
 0001:00001f28       ??_C@_1FC@OJGKKKJI@?$AAR?$AAe?$AAp?$AAe?$AAa?$AAt?$AAe?$AAd?$AAS?$AAt?$AAa?$AAr?$AAt?$AA?3?$AA?5?$AAM?$AAa?$AAs?$AAt?$AAe?$AAr?$AA?5?$AAm?$AAo?$AAd?$AAe?$AA?5?$AAs?$AAe?$AAt?$AA?5?$AAf@ 10002f28     i2c_mx25_topaz_v1:i2cClass.obj
 0001:00001f80       ??_C@_1EM@FDMACOMC@?$AAI?$AAA?$AAL?$AA?5?$AAd?$AAe?$AAt?$AAe?$AAc?$AAt?$AA?5?$AAi?$AAn?$AA?5?$AAG?$AAe?$AAn?$AAe?$AAr?$AAa?$AAt?$AAe?$AAR?$AAe?$AAp?$AAe?$AAa?$AAt?$AAe?$AAd?$AAS?$AAt@ 10002f80     i2c_mx25_topaz_v1:i2cClass.obj
 0001:00001fcc       ??_C@_1CG@DCOMGPKI@?$AAS?$AAR?$AA?$DN?$AA?$CF?$AA0?$AA2?$AAx?$AA?0?$AA?5?$AAC?$AAR?$AA?$DN?$AA?$CF?$AA0?$AA2?$AAx?$AA?$AN?$AA?6?$AA?$AA@ 10002fcc     i2c_mx25_topaz_v1:i2cClass.obj
 0001:00001ff4       ??_C@_1DI@OICKEDCO@?$AAG?$AAe?$AAn?$AAe?$AAr?$AAa?$AAt?$AAe?$AAS?$AAt?$AAo?$AAp?$AA?5?$AAn?$AAo?$AAt?$AA?5?$AAc?$AAo?$AAm?$AAp?$AAl?$AAe?$AAt?$AAe?$AA?$AN?$AA?6?$AA?$AA@ 10002ff4     i2c_mx25_topaz_v1:i2cClass.obj
 0001:00002030       ??_C@_1EM@CLABPHNM@?$AAM?$AAS?$AAT?$AAA?$AA?5?$AAn?$AAo?$AAt?$AA?5?$AAs?$AAe?$AAt?$AA?5?$AAd?$AAe?$AAt?$AAe?$AAc?$AAt?$AA?5?$AAi?$AAn?$AA?5?$AAG?$AAe?$AAn?$AAe?$AAr?$AAa?$AAt?$AAe?$AAS@ 10003030     i2c_mx25_topaz_v1:i2cClass.obj
 0001:0000207c       ??_C@_1DK@PBMPABKH@?$AAI?$AAA?$AAL?$AA?5?$AAd?$AAe?$AAt?$AAe?$AAc?$AAt?$AA?5?$AAi?$AAn?$AA?5?$AAG?$AAe?$AAn?$AAe?$AAr?$AAa?$AAt?$AAe?$AAS?$AAt?$AAo?$AAp?$AA?$AN?$AA?6?$AA?$AA@ 1000307c     i2c_mx25_topaz_v1:i2cClass.obj
 0001:000020b8       ??_C@_1GA@FHENJBBP@?$AAW?$AAa?$AAr?$AAn?$AAi?$AAn?$AAg?$AA?3?$AA?5?$AAE?$AAv?$AAe?$AAn?$AAt?$AA?5?$AAr?$AAe?$AAm?$AAa?$AAi?$AAn?$AA?5?$AAA?$AAF?$AAT?$AAE?$AAR?$AA?5?$AAW?$AAr?$AAi?$AAt@ 100030b8     i2c_mx25_topaz_v1:i2cClass.obj
 0001:00002118       ??_C@_1JG@BOHDDOCN@?$AAI?$AA2?$AAC?$AAC?$AAl?$AAa?$AAs?$AAs?$AA?3?$AA?3?$AAP?$AAr?$AAo?$AAc?$AAe?$AAs?$AAs?$AAP?$AAa?$AAc?$AAk?$AAe?$AAt?$AA?$CI?$AA?$CJ?$AA?3?$AA?5?$AAS?$AAe?$AAn?$AAd?$AA?5@ 10003118     i2c_mx25_topaz_v1:i2cClass.obj
 0001:000021b0       ??_C@_1DO@PEBFECGE@?$AAI?$AAI?$AAF?$AA?5?$AAd?$AAo?$AAs?$AAe?$AA?5?$AAn?$AAo?$AAt?$AA?5?$AAr?$AAe?$AAs?$AAe?$AAt?$AA?5?$AAi?$AAn?$AA?5?$AAW?$AAR?$AA?4?$AAP?$AAk?$AAt?$AA?$AN?$AA?6?$AA?$AA@ 100031b0     i2c_mx25_topaz_v1:i2cClass.obj
 0001:000021f0       ??_C@_1GI@EEKNOBBN@?$AAI?$AA2?$AAC?$AAC?$AAl?$AAa?$AAs?$AAs?$AA?3?$AA?3?$AAP?$AAr?$AAo?$AAc?$AAe?$AAs?$AAs?$AAP?$AAa?$AAc?$AAk?$AAe?$AAt?$AA?$CI?$AA?$CJ?$AA?3?$AA?5?$AAN?$AAo?$AA?5?$AAA?$AAC@ 100031f0     i2c_mx25_topaz_v1:i2cClass.obj
 0001:00002258       ??_C@_1FM@GHADEGC@?$AAI?$AA2?$AAC?$AAC?$AAl?$AAa?$AAs?$AAs?$AA?3?$AA?3?$AAP?$AAr?$AAo?$AAc?$AAe?$AAs?$AAs?$AAP?$AAa?$AAc?$AAk?$AAe?$AAt?$AA?$CI?$AA?$CJ?$AA?3?$AA?5?$AAG?$AAo?$AAt?$AA?5?$AAD@ 10003258     i2c_mx25_topaz_v1:i2cClass.obj
 0001:000022b8       ??_C@_1FO@JIAIPJAA@?$AAI?$AA2?$AAC?$AAC?$AAl?$AAa?$AAs?$AAs?$AA?3?$AA?3?$AAP?$AAr?$AAo?$AAc?$AAe?$AAs?$AAs?$AAP?$AAa?$AAc?$AAk?$AAe?$AAt?$AA?$CI?$AA?$CJ?$AA?3?$AA?5?$AAC?$AAl?$AAe?$AAa?$AAr@ 100032b8     i2c_mx25_topaz_v1:i2cClass.obj
 0001:00002318       ??_C@_1EM@DLALMNHC@?$AAD?$AAo?$AAw?$AAn?$AA?5?$AAg?$AAr?$AAa?$AAd?$AAe?$AA?5?$AAi?$AA2?$AAc?$AA?5?$AAt?$AAo?$AA?5?$AAp?$AAo?$AAl?$AAl?$AAi?$AAn?$AAg?$AA?5?$AAm?$AAo?$AAd?$AAe?$AA?4?$AA?$CI@ 10003318     i2c_mx25_topaz_v1:i2cClass.obj
 0001:00002368       ??_C@_1EK@JDIFLNF@?$AAD?$AAo?$AAw?$AAn?$AA?5?$AAg?$AAr?$AAa?$AAd?$AAe?$AA?5?$AAi?$AA2?$AAc?$AA?5?$AAt?$AAo?$AA?5?$AAp?$AAo?$AAl?$AAl?$AAi?$AAn?$AAg?$AA?5?$AAm?$AAo?$AAd?$AAe?$AA?4?$AA?$CI@ 10003368     i2c_mx25_topaz_v1:i2cClass.obj
 0001:000023b8       ??_C@_1HE@LCELACHJ@?$AAI?$AA2?$AAC?$AAC?$AAl?$AAa?$AAs?$AAs?$AA?3?$AA?3?$AAP?$AAr?$AAo?$AAc?$AAe?$AAs?$AAs?$AAP?$AAa?$AAc?$AAk?$AAe?$AAt?$AA?$CI?$AA?$CJ?$AA?3?$AA?5?$AAT?$AAr?$AAa?$AAn?$AAs@ 100033b8     i2c_mx25_topaz_v1:i2cClass.obj
 0001:00002430       ??_C@_1GO@JKAGFKID@?$AAW?$AAa?$AAr?$AAn?$AAi?$AAn?$AAg?$AA?3?$AA?5?$AAE?$AAv?$AAe?$AAn?$AAt?$AA?5?$AAr?$AAe?$AAm?$AAa?$AAi?$AAn?$AA?5?$AAp?$AAe?$AAn?$AAd?$AAi?$AAn?$AAg?$AA?5?$AAA?$AAF@ 10003430     i2c_mx25_topaz_v1:i2cClass.obj
 0001:000024a0       ??_C@_1FI@PLOLLODP@?$AAI?$AA2?$AAC?$AAC?$AAl?$AAa?$AAs?$AAs?$AA?3?$AA?3?$AAP?$AAr?$AAo?$AAc?$AAe?$AAs?$AAs?$AAP?$AAa?$AAc?$AAk?$AAe?$AAt?$AA?$CI?$AA?$CJ?$AA?3?$AA?5?$AAB?$AAy?$AAt?$AAe?$AA?5@ 100034a0     i2c_mx25_topaz_v1:i2cClass.obj
 0001:000024f8       ??_C@_1FM@BACKNOHL@?$AAI?$AA2?$AAC?$AAC?$AAl?$AAa?$AAs?$AAs?$AA?3?$AA?3?$AAP?$AAr?$AAo?$AAc?$AAe?$AAs?$AAs?$AAP?$AAa?$AAc?$AAk?$AAe?$AAt?$AA?$CI?$AA?$CJ?$AA?3?$AA?5?$AAR?$AAe?$AAa?$AAd?$AA?5@ 100034f8     i2c_mx25_topaz_v1:i2cClass.obj
 0001:00002558       ??_C@_1JA@FGLJIAHP@?$AAI?$AA2?$AAC?$AAC?$AAl?$AAa?$AAs?$AAs?$AA?3?$AA?3?$AAP?$AAr?$AAo?$AAc?$AAe?$AAs?$AAs?$AAP?$AAa?$AAc?$AAk?$AAe?$AAt?$AA?$CI?$AA?$CJ?$AA?3?$AA?5?$AAS?$AAe?$AAn?$AAd?$AA?5@ 10003558     i2c_mx25_topaz_v1:i2cClass.obj
 0001:000025e8       ??_C@_1HM@KHHFDMBB@?$AAI?$AA2?$AAC?$AAC?$AAl?$AAa?$AAs?$AAs?$AA?3?$AA?3?$AAP?$AAr?$AAo?$AAc?$AAe?$AAs?$AAs?$AAP?$AAa?$AAc?$AAk?$AAe?$AAt?$AA?$CI?$AA?$CJ?$AA?3?$AA?5?$AAC?$AAh?$AAa?$AAn?$AAg@ 100035e8     i2c_mx25_topaz_v1:i2cClass.obj
 0001:00002668       ??_C@_1IE@ENMKMKON@?$AAI?$AA2?$AAC?$AAC?$AAl?$AAa?$AAs?$AAs?$AA?3?$AA?3?$AAP?$AAr?$AAo?$AAc?$AAe?$AAs?$AAs?$AAP?$AAa?$AAc?$AAk?$AAe?$AAt?$AA?$CI?$AA?$CJ?$AA?3?$AA?5?$AAi?$AAn?$AAt?$AAe?$AAr@ 10003668     i2c_mx25_topaz_v1:i2cClass.obj
 0001:000026f0       ??_C@_1EM@KDKILKGC@?$AAD?$AAo?$AAw?$AAn?$AA?5?$AAg?$AAr?$AAa?$AAd?$AAe?$AA?5?$AAi?$AA2?$AAc?$AA?5?$AAt?$AAo?$AA?5?$AAp?$AAo?$AAl?$AAl?$AAi?$AAn?$AAg?$AA?5?$AAm?$AAo?$AAd?$AAe?$AA?4?$AA?$CI@ 100036f0     i2c_mx25_topaz_v1:i2cClass.obj
 0001:00002740       ??_C@_1EK@OPBBJAJB@?$AAD?$AAo?$AAw?$AAn?$AA?5?$AAg?$AAr?$AAa?$AAd?$AAe?$AA?5?$AAi?$AA2?$AAc?$AA?5?$AAt?$AAo?$AA?5?$AAp?$AAo?$AAl?$AAl?$AAi?$AAn?$AAg?$AA?5?$AAm?$AAo?$AAd?$AAe?$AA?4?$AA?$CI@ 10003740     i2c_mx25_topaz_v1:i2cClass.obj
 0001:00002790       ??_C@_1IO@FPJFBKEP@?$AAI?$AA2?$AAC?$AAC?$AAl?$AAa?$AAs?$AAs?$AA?3?$AA?3?$AAP?$AAr?$AAo?$AAc?$AAe?$AAs?$AAs?$AAP?$AAa?$AAc?$AAk?$AAe?$AAt?$AA?$CI?$AA?$CJ?$AA?3?$AA?5?$AAD?$AAu?$AAm?$AAm?$AAy@ 10003790     i2c_mx25_topaz_v1:i2cClass.obj
 0001:00002820       ??_C@_1GG@KHJEDHDO@?$AAI?$AA2?$AAC?$AAC?$AAl?$AAa?$AAs?$AAs?$AA?3?$AA?3?$AAP?$AAr?$AAo?$AAc?$AAe?$AAs?$AAs?$AAP?$AAa?$AAc?$AAk?$AAe?$AAt?$AA?$CI?$AA?$CJ?$AA?3?$AA?5?$AAD?$AAi?$AAs?$AAa?$AAb@ 10003820     i2c_mx25_topaz_v1:i2cClass.obj
 0001:00002888       ??_C@_1EG@GCIPGBI@?$AAI?$AAI?$AAF?$AA?5?$AAd?$AAo?$AAs?$AAe?$AA?5?$AAn?$AAo?$AAt?$AA?5?$AAr?$AAe?$AAs?$AAe?$AAt?$AA?5?$AAi?$AAn?$AA?5?$AAP?$AAr?$AAo?$AAc?$AAe?$AAs?$AAs?$AAP?$AAk?$AAt@ 10003888     i2c_mx25_topaz_v1:i2cClass.obj
 0001:000028d0       ??_C@_1GE@OHLDAJHI@?$AAI?$AA2?$AAC?$AAC?$AAl?$AAa?$AAs?$AAs?$AA?3?$AA?3?$AAP?$AAr?$AAo?$AAc?$AAe?$AAs?$AAs?$AAP?$AAa?$AAc?$AAk?$AAe?$AAt?$AA?$CI?$AA?$CJ?$AA?3?$AA?5?$AAI?$AA2?$AAC?$AA?5?$AAI@ 100038d0     i2c_mx25_topaz_v1:i2cClass.obj
 0001:00002938       ??_C@_1HI@PJJGMPBJ@?$AAI?$AA2?$AAC?$AAC?$AAl?$AAa?$AAs?$AAs?$AA?3?$AA?3?$AAP?$AAr?$AAo?$AAc?$AAe?$AAs?$AAs?$AAP?$AAa?$AAc?$AAk?$AAe?$AAt?$AA?$CI?$AA?$CJ?$AA?3?$AAI?$AAs?$AAs?$AAu?$AAi?$AAn@ 10003938     i2c_mx25_topaz_v1:i2cClass.obj
 0001:000029b0       ??_C@_1GG@MEDJEENI@?$AAI?$AA2?$AAC?$AAC?$AAl?$AAa?$AAs?$AAs?$AA?3?$AA?3?$AAP?$AAr?$AAo?$AAc?$AAe?$AAs?$AAs?$AAP?$AAa?$AAc?$AAk?$AAe?$AAt?$AA?$CI?$AA?$CJ?$AA?3?$AAI?$AAs?$AAs?$AAu?$AAi?$AAn@ 100039b0     i2c_mx25_topaz_v1:i2cClass.obj
 0001:00002a18       ??_C@_1IA@CPCAJKAF@?$AAI?$AA2?$AAC?$AAC?$AAl?$AAa?$AAs?$AAs?$AA?3?$AA?3?$AAP?$AAr?$AAo?$AAc?$AAe?$AAs?$AAs?$AAP?$AAa?$AAc?$AAk?$AAe?$AAt?$AA?$CI?$AA?$CJ?$AA?3?$AA?5?$AAS?$AAe?$AAt?$AAt?$AAi@ 10003a18     i2c_mx25_topaz_v1:i2cClass.obj
 0001:00002a98       ??_C@_1GG@KPFCHIKN@?$AAI?$AA2?$AAC?$AAC?$AAl?$AAa?$AAs?$AAs?$AA?3?$AA?3?$AAP?$AAr?$AAo?$AAc?$AAe?$AAs?$AAs?$AAP?$AAa?$AAc?$AAk?$AAe?$AAt?$AA?$CI?$AA?$CJ?$AA?3?$AA?5?$AAE?$AAn?$AAa?$AAb?$AAl@ 10003a98     i2c_mx25_topaz_v1:i2cClass.obj
 0001:00002b00       ??_C@_1FC@PBACOMHC@?$AAI?$AA2?$AAC?$AAC?$AAl?$AAa?$AAs?$AAs?$AA?3?$AA?3?$AAP?$AAr?$AAo?$AAc?$AAe?$AAs?$AAs?$AAP?$AAa?$AAc?$AAk?$AAe?$AAt?$AA?$CI?$AA?$CJ?$AA?3?$AA?5?$AAE?$AAn?$AAa?$AAb?$AAl@ 10003b00     i2c_mx25_topaz_v1:i2cClass.obj
 0001:00002b58       ??_C@_1HG@MHKLNKKC@?$AAI?$AA2?$AAC?$AAC?$AAl?$AAa?$AAs?$AAs?$AA?3?$AA?3?$AAP?$AAr?$AAo?$AAc?$AAe?$AAs?$AAs?$AAP?$AAa?$AAc?$AAk?$AAe?$AAt?$AA?$CI?$AA?$CJ?$AA?3?$AA?5?$AAC?$AAo?$AAn?$AAf?$AAi@ 10003b58     i2c_mx25_topaz_v1:i2cClass.obj
 0001:00002bd0       ??_C@_1FM@HCIKHFCM@?$AAI?$AA2?$AAC?$AAC?$AAl?$AAa?$AAs?$AAs?$AA?3?$AA?3?$AAP?$AAr?$AAo?$AAc?$AAe?$AAs?$AAs?$AAP?$AAa?$AAc?$AAk?$AAe?$AAt?$AA?$CI?$AA?$CJ?$AA?3?$AA?5?$AAS?$AAe?$AAt?$AA?5?$AAI@ 10003bd0     i2c_mx25_topaz_v1:i2cClass.obj
 0001:00002c30       ??_C@_1HA@NIPALFN@?$AAI?$AA2?$AAC?$AAC?$AAl?$AAa?$AAs?$AAs?$AA?3?$AA?3?$AAP?$AAr?$AAo?$AAc?$AAe?$AAs?$AAs?$AAP?$AAa?$AAc?$AAk?$AAe?$AAt?$AA?$CI?$AA?$CJ?$AA?3?$AA?5?$AAT?$AAr?$AAy?$AAi?$AAn@ 10003c30     i2c_mx25_topaz_v1:i2cClass.obj
 0001:00002ca0       ??_C@_1FK@MKCJKADI@?$AAI?$AA2?$AAC?$AAC?$AAl?$AAa?$AAs?$AAs?$AA?3?$AA?3?$AAP?$AAr?$AAo?$AAc?$AAe?$AAs?$AAs?$AAP?$AAa?$AAc?$AAk?$AAe?$AAt?$AA?$CI?$AA?$CJ?$AA?3?$AA?5?$AAR?$AAe?$AAs?$AAe?$AAt@ 10003ca0     i2c_mx25_topaz_v1:i2cClass.obj
 0001:00002d00       ??_C@_1FK@LOLBEJLH@?$AAI?$AA2?$AAC?$AAC?$AAl?$AAa?$AAs?$AAs?$AA?3?$AA?3?$AAP?$AAr?$AAo?$AAc?$AAe?$AAs?$AAs?$AAP?$AAa?$AAc?$AAk?$AAe?$AAt?$AA?$CI?$AA?$CJ?$AA?3?$AA?5?$AAR?$AAe?$AAs?$AAe?$AAt@ 10003d00     i2c_mx25_topaz_v1:i2cClass.obj
 0001:00002d60       ??_C@_1JE@EKIDKDIB@?$AAI?$AA2?$AAC?$AAC?$AAl?$AAa?$AAs?$AAs?$AA?3?$AA?3?$AAP?$AAr?$AAo?$AAc?$AAe?$AAs?$AAs?$AAP?$AAa?$AAc?$AAk?$AAe?$AAt?$AA?$CI?$AA?$CJ?$AA?3?$AAI?$AA2?$AAC?$AA?5?$AAB?$AAu@ 10003d60     i2c_mx25_topaz_v1:i2cClass.obj
 0001:00002df8       ??_C@_1JO@DILLLDOI@?$AAI?$AA2?$AAC?$AAC?$AAl?$AAa?$AAs?$AAs?$AA?3?$AA?3?$AAP?$AAr?$AAo?$AAc?$AAe?$AAs?$AAs?$AAP?$AAa?$AAc?$AAk?$AAe?$AAt?$AA?$CI?$AA?$CJ?$AA?3?$AAB?$AAS?$AAP?$AAI?$AA2?$AAC@ 10003df8     i2c_mx25_topaz_v1:i2cClass.obj
 0001:00002e98       ??_C@_1IM@CEMCLNGE@?$AAI?$AA2?$AAC?$AAC?$AAl?$AAa?$AAs?$AAs?$AA?3?$AA?3?$AAP?$AAr?$AAo?$AAc?$AAe?$AAs?$AAs?$AAP?$AAa?$AAc?$AAk?$AAe?$AAt?$AA?$CI?$AA?$CJ?$AA?3?$AAB?$AAS?$AAP?$AAI?$AA2?$AAC@ 10003e98     i2c_mx25_topaz_v1:i2cClass.obj
 0001:00002f28       ??_C@_1GI@HGKCPGFG@?$AAI?$AA2?$AAC?$AAC?$AAl?$AAa?$AAs?$AAs?$AA?3?$AA?3?$AAP?$AAr?$AAo?$AAc?$AAe?$AAs?$AAs?$AAP?$AAa?$AAc?$AAk?$AAe?$AAt?$AA?$CI?$AA?$CJ?$AA?3?$AA?5?$AAA?$AAc?$AAq?$AAu?$AAi@ 10003f28     i2c_mx25_topaz_v1:i2cClass.obj
 0001:00002f90       ??_C@_1GM@IKJHBEAH@?$AAI?$AA2?$AAC?$AAC?$AAl?$AAa?$AAs?$AAs?$AA?3?$AA?3?$AAP?$AAr?$AAo?$AAc?$AAe?$AAs?$AAs?$AAP?$AAa?$AAc?$AAk?$AAe?$AAt?$AA?$CI?$AA?$CJ?$AA?3?$AA?5?$AAW?$AAa?$AAi?$AAt?$AAi@ 10003f90     i2c_mx25_topaz_v1:i2cClass.obj
 0001:00002ffc       ??_C@_1BO@MJJAIOPJ@?$AA?$CF?$AAs?$AA?3?$AA?5?$AAT?$AAi?$AAm?$AAe?$AA?5?$AAo?$AAu?$AAt?$AA?$AN?$AA?6?$AA?$AA@ 10003ffc     i2c_mx25_topaz_v1:i2cClass.obj
 0001:0000301c       ??_C@_1DG@JJMEANOC@?$AAi?$AAn?$AAt?$AAe?$AAr?$AAr?$AAu?$AAp?$AAt?$AA?5?$AAe?$AAv?$AAe?$AAn?$AAt?$AA?5?$AAd?$AAi?$AAs?$AAc?$AAa?$AAr?$AAd?$AA?4?$AA?$AN?$AA?6?$AA?$AA@ 1000401c     i2c_mx25_topaz_v1:i2cClass.obj
 0001:00003054       ??_C@_1DC@IBOEJLKK@?$AA?$CF?$AAs?$AA?3?$AA?5?$AAI?$AAn?$AAt?$AAe?$AAr?$AAr?$AAu?$AAp?$AAt?$AA?5?$AAr?$AAe?$AAc?$AAe?$AAi?$AAv?$AAe?$AAd?$AA?$AN?$AA?6?$AA?$AA@ 10004054     i2c_mx25_topaz_v1:i2cClass.obj
 0001:00003088       ??_C@_1CE@KFJAIJEG@?$AA?$CF?$AAs?$AA?3?$AA?5?$AAI?$AAn?$AA?5?$AAt?$AAh?$AAe?$AA?5?$AAl?$AAo?$AAo?$AAp?$AA?$AN?$AA?6?$AA?$AA@ 10004088     i2c_mx25_topaz_v1:i2cClass.obj
 0001:000030ac       ??_C@_1DM@ICFJNPCP@?$AAI?$AA2?$AAC?$AAC?$AAl?$AAa?$AAs?$AAs?$AA?3?$AA?3?$AAI?$AA2?$AAC?$AAI?$AAn?$AAt?$AAe?$AAr?$AAr?$AAu?$AAp?$AAt?$AAH?$AAa?$AAn?$AAd?$AAl?$AAe?$AAr?$AA?$AA@ 100040ac     i2c_mx25_topaz_v1:i2cClass.obj
 0001:000030e8       ??_C@_1FC@LFKGMLNJ@?$AAI?$AA2?$AAC?$AAC?$AAl?$AAa?$AAs?$AAs?$AA?3?$AA?3?$AAE?$AAn?$AAa?$AAb?$AAl?$AAe?$AAS?$AAl?$AAa?$AAv?$AAe?$AA?$CI?$AA?$CJ?$AA?3?$AA?5?$AAR?$AAe?$AA?5?$AAi?$AAn?$AAi?$AAt@ 100040e8     i2c_mx25_topaz_v1:i2cClass.obj
 0001:00003140       ??_C@_1EE@LLDBDOHL@?$AAI?$AA2?$AAC?$AAC?$AAl?$AAa?$AAs?$AAs?$AA?3?$AA?3?$AAD?$AAi?$AAs?$AAa?$AAb?$AAl?$AAe?$AAS?$AAl?$AAa?$AAv?$AAe?$AA?$CI?$AA?$CJ?$AA?3?$AA?5?$AAI?$AA2?$AAC?$AAR?$AA?5?$AA?$AN@ 10004140     i2c_mx25_topaz_v1:i2cClass.obj
 0001:000031a4       BSPI2CGetModuleClock       100041a4 f   bspi2c.obj
 0001:000031e0       BSPI2CIOMUXConfig          100041e0 f   bspi2c.obj
 0001:000033e4       BSPI2CEnableClock          100043e4 f   bspi2c.obj
 0001:000034fc       BSPGetTimeoutValue         100044fc f   bspi2c.obj
 0001:00003514       ?I2C_Init@@YAKPBG@Z        10004514 f   i2c_mx25_topaz_v1:i2c_io.obj
 0001:0000385c       ?I2C_Deinit@@YAHK@Z        1000485c f   i2c_mx25_topaz_v1:i2c_io.obj
 0001:0000395c       ?I2C_Open@@YAKKKK@Z        1000495c f   i2c_mx25_topaz_v1:i2c_io.obj
 0001:00003a08       ?I2C_Close@@YAHK@Z         10004a08 f   i2c_mx25_topaz_v1:i2c_io.obj
 0001:00003ab0       ?I2C_PowerDown@@YAXK@Z     10004ab0 f   i2c_mx25_topaz_v1:i2c_io.obj
 0001:00003ac0       ?I2C_PowerUp@@YAXXZ        10004ac0 f   i2c_mx25_topaz_v1:i2c_io.obj
 0001:00003ac4       ?I2C_Read@@YAKKPAXK@Z      10004ac4 f   i2c_mx25_topaz_v1:i2c_io.obj
 0001:00003ae8       ?I2C_Write@@YAKKPBXK@Z     10004ae8 f   i2c_mx25_topaz_v1:i2c_io.obj
 0001:00003b0c       ?I2C_Seek@@YAKKJG@Z        10004b0c f   i2c_mx25_topaz_v1:i2c_io.obj
 0001:00003b38       ?I2C_IOControl@@YAHKKPAEK0KPAK@Z 10004b38 f   i2c_mx25_topaz_v1:i2c_io.obj
 0001:00005174       ?I2C_DllEntry@@YAHPAXK0@Z  10006174 f   i2c_mx25_topaz_v1:i2c_io.obj
 0001:00005240       ?IsLastActionOK@I2CClass@@QAAHXZ 10006240 f i i2c_mx25_topaz_v1:i2c_io.obj
 0001:0000528c       ?GetLastResult@I2CClass@@QAAHXZ 1000628c f i i2c_mx25_topaz_v1:i2c_io.obj
 0001:000052b8       ?SetSlaveBuf@I2CClass@@QAAPAUtagI2CSLAVEBUF@@PAU2@@Z 100062b8 f i i2c_mx25_topaz_v1:i2c_io.obj
 0001:000052fc       ??_GI2CClass@@QAAPAXI@Z    100062fc f i i2c_mx25_topaz_v1:i2c_io.obj
 0001:0000533c       ?GetClockRateDivider@I2CClass@@QAAGXZ 1000633c f i i2c_mx25_topaz_v1:i2c_io.obj
 0001:00005368       ?SetClockRateDivider@I2CClass@@QAAGG@Z 10006368 f i i2c_mx25_topaz_v1:i2c_io.obj
 0001:000053a4       ?GetSelfAddress@I2CClass@@QAAEXZ 100063a4 f i i2c_mx25_topaz_v1:i2c_io.obj
 0001:000053d0       ?SetSelfAddress@I2CClass@@QAAEE@Z 100063d0 f i i2c_mx25_topaz_v1:i2c_io.obj
 0001:0000540c       ?GetMode@I2CClass@@QAAEXZ  1000640c f i i2c_mx25_topaz_v1:i2c_io.obj
 0001:00005438       ?SetMode@I2CClass@@QAAEE@Z 10006438 f i i2c_mx25_topaz_v1:i2c_io.obj
 0001:00005474       ??1MarshalledBuffer_t@@QAA@XZ 10006474 f i i2c_mx25_topaz_v1:i2c_io.obj
 0001:0000548c       ??0MarshalledBuffer_t@@QAA@PAXKKHH@Z 1000648c f i i2c_mx25_topaz_v1:i2c_io.obj
 0001:000054dc       ?Reset@MarshalledBuffer_t@@AAAXXZ 100064dc f i i2c_mx25_topaz_v1:i2c_io.obj
 0001:00005518       ?Marshal@MarshalledBuffer_t@@QAAJPAXKKHH@Z 10006518 f i i2c_mx25_topaz_v1:i2c_io.obj
 0001:00005618       ?Unmarshal@MarshalledBuffer_t@@QAAJXZ 10006618 f i i2c_mx25_topaz_v1:i2c_io.obj
 0001:000056e4       ?ptr@MarshalledBuffer_t@@QBAPAXXZ 100066e4 f i i2c_mx25_topaz_v1:i2c_io.obj
 0001:00005730       ??_GMarshalledBuffer_t@@QAAPAXI@Z 10006730 f i i2c_mx25_topaz_v1:i2c_io.obj
 0001:00005770       ??0?$Buffer_t@VDuplicateTraits_t@detail@marshal@ce@@@detail@marshal@ce@@QAA@PAXKK@Z 10006770 f i i2c_mx25_topaz_v1:i2c_io.obj
 0001:000057c0       ?ptr@?$Buffer_t@VDuplicateTraits_t@detail@marshal@ce@@@detail@marshal@ce@@QBAPAXXZ 100067c0 f i i2c_mx25_topaz_v1:i2c_io.obj
 0001:000057ec       ??1?$Buffer_t@VDuplicateTraits_t@detail@marshal@ce@@@detail@marshal@ce@@UAA@XZ 100067ec f i i2c_mx25_topaz_v1:i2c_io.obj
 0001:00005814       ??_G?$Buffer_t@VDuplicateTraits_t@detail@marshal@ce@@@detail@marshal@ce@@UAAPAXI@Z 10006814 f i i2c_mx25_topaz_v1:i2c_io.obj
 0001:00005814       ??_E?$Buffer_t@VDuplicateTraits_t@detail@marshal@ce@@@detail@marshal@ce@@UAAPAXI@Z 10006814 f i i2c_mx25_topaz_v1:i2c_io.obj
 0001:00005854       ?Reset@?$Buffer_t@VDuplicateTraits_t@detail@marshal@ce@@@detail@marshal@ce@@AAAXXZ 10006854 f i i2c_mx25_topaz_v1:i2c_io.obj
 0001:00005894       ?Free@?$Buffer_t@VDuplicateTraits_t@detail@marshal@ce@@@detail@marshal@ce@@QAAJXZ 10006894 f i i2c_mx25_topaz_v1:i2c_io.obj
 0001:0000592c       ?free@DuplicateTraits_t@detail@marshal@ce@@QBAJPAX0KK@Z 1000692c f i i2c_mx25_topaz_v1:i2c_io.obj
 0001:00005968       ?Allocate@?$Buffer_t@VDuplicateTraits_t@detail@marshal@ce@@@detail@marshal@ce@@QAAJPAXKK@Z 10006968 f i i2c_mx25_topaz_v1:i2c_io.obj
 0001:00005a18       ?alloc@DuplicateTraits_t@detail@marshal@ce@@QBAJPAPAXPAXKK@Z 10006a18 f i i2c_mx25_topaz_v1:i2c_io.obj
 0001:00005a54       ?CalculateClkRateDiv@I2CClass@@QAAGK@Z 10006a54 f   i2c_mx25_topaz_v1:i2cClass.obj
 0001:00005d44       ??0I2CClass@@QAA@I@Z       10006d44 f   i2c_mx25_topaz_v1:i2cClass.obj
 0001:000067b4       ??1I2CClass@@QAA@XZ        100077b4 f   i2c_mx25_topaz_v1:i2cClass.obj
 0001:00006adc       ?Reset@I2CClass@@QAAXXZ    10007adc f   i2c_mx25_topaz_v1:i2cClass.obj
 0001:00006b14       ?GenerateStart@I2CClass@@AAAHPAUI2C_PACKET@@@Z 10007b14 f   i2c_mx25_topaz_v1:i2cClass.obj
 0001:0000752c       ?GenerateRepeatedStart@I2CClass@@AAAHPAUI2C_PACKET@@H@Z 1000852c f   i2c_mx25_topaz_v1:i2cClass.obj
 0001:00007ed0       ?GenerateStop@I2CClass@@AAAXXZ 10008ed0 f   i2c_mx25_topaz_v1:i2cClass.obj
 0001:00008388       ?WritePacket@I2CClass@@AAAHPAUI2C_PACKET@@H@Z 10009388 f   i2c_mx25_topaz_v1:i2cClass.obj
 0001:00008c9c       ?ReadPacket@I2CClass@@AAAHPAUI2C_PACKET@@HHPAH@Z 10009c9c f   i2c_mx25_topaz_v1:i2cClass.obj
 0001:00009890       ?CleanupPendingInterrupt@I2CClass@@AAAHXZ 1000a890 f   i2c_mx25_topaz_v1:i2cClass.obj
 0001:00009948       ?ProcessPackets@I2CClass@@QAAHQAUI2C_PACKET@@H@Z 1000a948 f   i2c_mx25_topaz_v1:i2cClass.obj
 0001:0000a308       ?I2CIST@I2CClass@@CAXPAX@Z 1000b308 f   i2c_mx25_topaz_v1:i2cClass.obj
 0001:0000a334       ?I2CInterruptHandler@I2CClass@@AAAXI@Z 1000b334 f   i2c_mx25_topaz_v1:i2cClass.obj
 0001:0000b0ec       ?RealMode@I2CClass@@QAAEXZ 1000c0ec f   i2c_mx25_topaz_v1:i2cClass.obj
 0001:0000b144       ?EnableSlave@I2CClass@@QAAHXZ 1000c144 f   i2c_mx25_topaz_v1:i2cClass.obj
 0001:0000b328       ?DisableSlave@I2CClass@@QAAHXZ 1000c328 f   i2c_mx25_topaz_v1:i2cClass.obj
 0001:0000b46c       ?SetSlaveText@I2CClass@@QAAHPAEK@Z 1000c46c f   i2c_mx25_topaz_v1:i2cClass.obj
 0001:0000b524       ?GetSlaveText@I2CClass@@QAAHPAEKPAK@Z 1000c524 f   i2c_mx25_topaz_v1:i2cClass.obj
 0001:0000b600       ?SetSlaveSize@I2CClass@@QAAHPAEK@Z 1000c600 f   i2c_mx25_topaz_v1:i2cClass.obj
 0001:0000b6d0       ?GetSlaveSize@I2CClass@@QAAHPAEKPAK@Z 1000c6d0 f   i2c_mx25_topaz_v1:i2cClass.obj
 0001:0000b734       PulseEvent                 1000c734 f i i2c_mx25_topaz_v1:i2cClass.obj
 0001:0000b768       ResetEvent                 1000c768 f i i2c_mx25_topaz_v1:i2cClass.obj
 0001:0000b79c       SetEvent                   1000c79c f i i2c_mx25_topaz_v1:i2cClass.obj
 0001:0000b7d0       I2CGetBaseRegAddr          1000c7d0 f   i2c_mx25_topaz_v1:cspi2c.obj
 0001:0000b854       I2CGetIRQ                  1000c854 f   i2c_mx25_topaz_v1:cspi2c.obj
 0001:0000b8cc       NKDbgPrintfW               1000c8cc f   coredll:COREDLL.dll
 0001:0000b8dc       RegCloseKey                1000c8dc f   coredll:COREDLL.dll
 0001:0000b8ec       RegQueryValueExW           1000c8ec f   coredll:COREDLL.dll
 0001:0000b8fc       OpenDeviceKey              1000c8fc f   coredll:COREDLL.dll
 0001:0000b90c       CeAllocAsynchronousBuffer  1000c90c f   coredll:COREDLL.dll
 0001:0000b91c       CeOpenCallerBuffer         1000c91c f   coredll:COREDLL.dll
 0001:0000b92c       CeCloseCallerBuffer        1000c92c f   coredll:COREDLL.dll
 0001:0000b93c       CeFreeAsynchronousBuffer   1000c93c f   coredll:COREDLL.dll
 0001:0000b94c       DisableThreadLibraryCalls  1000c94c f   coredll:COREDLL.dll
 0001:0000b95c       RegisterDbgZones           1000c95c f   coredll:COREDLL.dll
 0001:0000b96c       CeFreeDuplicateBuffer      1000c96c f   coredll:COREDLL.dll
 0001:0000b97c       CeAllocDuplicateBuffer     1000c97c f   coredll:COREDLL.dll
 0001:0000b98c       CeSetThreadPriority        1000c98c f   coredll:COREDLL.dll
 0001:0000b99c       CreateThread               1000c99c f   coredll:COREDLL.dll
 0001:0000b9ac       InterruptInitialize        1000c9ac f   coredll:COREDLL.dll
 0001:0000b9bc       KernelIoControl            1000c9bc f   coredll:COREDLL.dll
 0001:0000b9cc       InitializeCriticalSection  1000c9cc f   coredll:COREDLL.dll
 0001:0000b9dc       CreateEventW               1000c9dc f   coredll:COREDLL.dll
 0001:0000b9ec       GetLastError               1000c9ec f   coredll:COREDLL.dll
 0001:0000b9fc       DeleteCriticalSection      1000c9fc f   coredll:COREDLL.dll
 0001:0000ba0c       CloseHandle                1000ca0c f   coredll:COREDLL.dll
 0001:0000ba1c       InterruptDisable           1000ca1c f   coredll:COREDLL.dll
 0001:0000ba2c       EventModify                1000ca2c f   coredll:COREDLL.dll
 0001:0000ba3c       InterruptDone              1000ca3c f   coredll:COREDLL.dll
 0001:0000ba4c       WaitForSingleObject        1000ca4c f   coredll:COREDLL.dll
 0001:0000ba5c       Sleep                      1000ca5c f   coredll:COREDLL.dll
 0001:0000ba6c       LeaveCriticalSection       1000ca6c f   coredll:COREDLL.dll
 0001:0000ba7c       EnterCriticalSection       1000ca7c f   coredll:COREDLL.dll
 0001:0000ba8c       TryEnterCriticalSection    1000ca8c f   coredll:COREDLL.dll
 0001:0000ba9c       MmMapIoSpace               1000ca9c f   ceddk:CEDDK.dll
 0001:0000baac       MmUnmapIoSpace             1000caac f   ceddk:CEDDK.dll
 0001:0000babc       StallExecution             1000cabc f   ceddk:CEDDK.dll
 0001:0000bacc       DDKClockGetFreq            1000cacc f   cspddk:CSPDDK.dll
 0001:0000badc       DDKIomuxSelectInput        1000cadc f   cspddk:CSPDDK.dll
 0001:0000baec       DDKIomuxSetPadConfig       1000caec f   cspddk:CSPDDK.dll
 0001:0000bafc       DDKIomuxSetPinMux          1000cafc f   cspddk:CSPDDK.dll
 0001:0000bb0c       DDKClockSetGatingMode      1000cb0c f   cspddk:CSPDDK.dll
 0001:0000bb1c       DllMain                    1000cb1c f   corelib0:dllmain.obj
 0001:0000bb54       _DllMainCRTStartup         1000cb54 f   corelib0:pegdmain.obj
 0001:0000bcec       __security_init_cookie     1000ccec f   corelib0:seccinit.obj
 0001:0000bd84       exit                       1000cd84 f   corelib0:cexit.obj
 0001:0000bea8       _exit                      1000cea8 f   corelib0:cexit.obj
 0001:0000bec8       _cexit                     1000cec8 f   corelib0:cexit.obj
 0001:0000bee0       _c_exit                    1000cee0 f   corelib0:cexit.obj
 0001:0000bef8       _initterm                  1000cef8 f   corelib0:crt0dat.obj
 0001:0000bf44       _cinit                     1000cf44 f   corelib0:crt0dat.obj
 0001:0000bf74       __crt_ExitProcess          1000cf74 f   corelib0:exitproc_proxy.obj
 0001:0000bfa0       GetCurrentProcess          1000cfa0 f i corelib0:exitproc_proxy.obj
 0001:0000bfb8       _onexit                    1000cfb8 f   corelib0:onexit.obj
 0001:0000c194       atexit                     1000d194 f   corelib0:onexit.obj
 0001:0000c1e4       ??2@YAPAXI@Z               1000d1e4 f   corelib1:COREDLL.dll
 0001:0000c1f4       ??3@YAXPAX@Z               1000d1f4 f   corelib1:COREDLL.dll
 0001:0000c204       memset                     1000d204 f   corelib1:COREDLL.dll
 0001:0000c214       __C_specific_handler       1000d214 f   corelib1:COREDLL.dll
 0001:0000c224       __rt_sdiv                  1000d224 f   corelib1:COREDLL.dll
 0001:0000c234       __rt_udiv                  1000d234 f   corelib1:COREDLL.dll
 0001:0000c244       memcpy                     1000d244 f   corelib1:COREDLL.dll
 0001:0000c254       _XcptFilter                1000d254 f   corelib1:COREDLL.dll
 0001:0000c264       __security_gen_cookie2     1000d264 f   corelib1:COREDLL.dll
 0001:0000c274       free                       1000d274 f   corelib1:COREDLL.dll
 0001:0000c284       realloc                    1000d284 f   corelib1:COREDLL.dll
 0001:0000c294       malloc                     1000d294 f   corelib1:COREDLL.dll
 0001:0000c2a4       _msize                     1000d2a4 f   corelib1:COREDLL.dll
 0001:0000c2b4       TerminateProcess           1000d2b4 f   coredll:COREDLL.dll
 0001:0000c30c       __IMPORT_DESCRIPTOR_COREDLL 1000d30c     coredll:COREDLL.dll
 0001:0000c320       __IMPORT_DESCRIPTOR_CEDDK  1000d320     ceddk:CEDDK.dll
 0001:0000c334       __IMPORT_DESCRIPTOR_CSPDDK 1000d334     cspddk:CSPDDK.dll
 0001:0000c348       __NULL_IMPORT_DESCRIPTOR   1000d348     coredll:COREDLL.dll
 0002:00000000       __imp_MmUnmapIoSpace       1000e000     ceddk:CEDDK.dll
 0002:00000004       __imp_MmMapIoSpace         1000e004     ceddk:CEDDK.dll
 0002:00000008       __imp_StallExecution       1000e008     ceddk:CEDDK.dll
 0002:0000000c       \177CEDDK_NULL_THUNK_DATA  1000e00c     ceddk:CEDDK.dll
 0002:00000010       __imp_CeAllocAsynchronousBuffer 1000e010     coredll:COREDLL.dll
 0002:00000014       __imp_CeOpenCallerBuffer   1000e014     coredll:COREDLL.dll
 0002:00000018       __imp_CeCloseCallerBuffer  1000e018     coredll:COREDLL.dll
 0002:0000001c       __imp_CeFreeAsynchronousBuffer 1000e01c     coredll:COREDLL.dll
 0002:00000020       __imp_DisableThreadLibraryCalls 1000e020     coredll:COREDLL.dll
 0002:00000024       __imp_RegisterDbgZones     1000e024     coredll:COREDLL.dll
 0002:00000028       __imp_CeFreeDuplicateBuffer 1000e028     coredll:COREDLL.dll
 0002:0000002c       __imp_CeAllocDuplicateBuffer 1000e02c     coredll:COREDLL.dll
 0002:00000030       __imp_CeSetThreadPriority  1000e030     coredll:COREDLL.dll
 0002:00000034       __imp_CreateThread         1000e034     coredll:COREDLL.dll
 0002:00000038       __imp_InterruptInitialize  1000e038     coredll:COREDLL.dll
 0002:0000003c       __imp_KernelIoControl      1000e03c     coredll:COREDLL.dll
 0002:00000040       __imp_OpenDeviceKey        1000e040     coredll:COREDLL.dll
 0002:00000044       __imp_CreateEventW         1000e044     coredll:COREDLL.dll
 0002:00000048       __imp_GetLastError         1000e048     coredll:COREDLL.dll
 0002:0000004c       __imp_DeleteCriticalSection 1000e04c     coredll:COREDLL.dll
 0002:00000050       __imp_CloseHandle          1000e050     coredll:COREDLL.dll
 0002:00000054       __imp_InterruptDisable     1000e054     coredll:COREDLL.dll
 0002:00000058       __imp_EventModify          1000e058     coredll:COREDLL.dll
 0002:0000005c       __imp_InterruptDone        1000e05c     coredll:COREDLL.dll
 0002:00000060       __imp_WaitForSingleObject  1000e060     coredll:COREDLL.dll
 0002:00000064       __imp_Sleep                1000e064     coredll:COREDLL.dll
 0002:00000068       __imp_LeaveCriticalSection 1000e068     coredll:COREDLL.dll
 0002:0000006c       __imp_EnterCriticalSection 1000e06c     coredll:COREDLL.dll
 0002:00000070       __imp_TryEnterCriticalSection 1000e070     coredll:COREDLL.dll
 0002:00000074       __imp_RegQueryValueExW     1000e074     coredll:COREDLL.dll
 0002:00000078       __imp_RegCloseKey          1000e078     coredll:COREDLL.dll
 0002:0000007c       __imp_InitializeCriticalSection 1000e07c     coredll:COREDLL.dll
 0002:00000080       __imp_NKDbgPrintfW         1000e080     coredll:COREDLL.dll
 0002:00000084       __imp__msize               1000e084     corelib1:COREDLL.dll
 0002:00000088       __imp_malloc               1000e088     corelib1:COREDLL.dll
 0002:0000008c       __imp_realloc              1000e08c     corelib1:COREDLL.dll
 0002:00000090       __imp_free                 1000e090     corelib1:COREDLL.dll
 0002:00000094       __imp___security_gen_cookie2 1000e094     corelib1:COREDLL.dll
 0002:00000098       __imp__XcptFilter          1000e098     corelib1:COREDLL.dll
 0002:0000009c       __imp_??2@YAPAXI@Z         1000e09c     corelib1:COREDLL.dll
 0002:000000a0       __imp_??3@YAXPAX@Z         1000e0a0     corelib1:COREDLL.dll
 0002:000000a4       __imp_memset               1000e0a4     corelib1:COREDLL.dll
 0002:000000a8       __imp___C_specific_handler 1000e0a8     corelib1:COREDLL.dll
 0002:000000ac       __imp___rt_sdiv            1000e0ac     corelib1:COREDLL.dll
 0002:000000b0       __imp___rt_udiv            1000e0b0     corelib1:COREDLL.dll
 0002:000000b4       __imp_memcpy               1000e0b4     corelib1:COREDLL.dll
 0002:000000b8       __imp_TerminateProcess     1000e0b8     coredll:COREDLL.dll
 0002:000000bc       \177COREDLL_NULL_THUNK_DATA 1000e0bc     coredll:COREDLL.dll
 0002:000000c0       __imp_DDKIomuxSetPinMux    1000e0c0     cspddk:CSPDDK.dll
 0002:000000c4       __imp_DDKIomuxSetPadConfig 1000e0c4     cspddk:CSPDDK.dll
 0002:000000c8       __imp_DDKIomuxSelectInput  1000e0c8     cspddk:CSPDDK.dll
 0002:000000cc       __imp_DDKClockGetFreq      1000e0cc     cspddk:CSPDDK.dll
 0002:000000d0       __imp_DDKClockSetGatingMode 1000e0d0     cspddk:CSPDDK.dll
 0002:000000d4       \177CSPDDK_NULL_THUNK_DATA 1000e0d4     cspddk:CSPDDK.dll
 0002:000000d8       dpCurSettings              1000e0d8     i2c_mx25_topaz_v1:i2c_io.obj
 0002:0000051c       __security_cookie          1000e51c     corelib0:seccinit.obj
 0002:00000520       __security_cookie_complement 1000e520     corelib0:seccinit.obj
 0002:00000524       _exitflag                  1000e524     corelib0:cexit.obj
 0002:00000528       __onexitend                1000e528     <common>
 0002:0000052c       __onexitbegin              1000e52c     <common>
 0002:00000530       _pRawDllMain               1000e530     <common>

 entry point at        0001:0000bb54

 Static symbols

 0001:0000bba4       _DllMainCRTStartupHelper   1000cba4 f   corelib0:pegdmain.obj
 0001:0000bda4       doexit                     1000cda4 f   corelib0:cexit.obj
